:0A13F60000010202030304040505D0
:1008FD00E4F515F514F513F512C20CC209C20BC2BD
:10090D000A121B25120E397E007F908E668F677539
:10091D006E00756FA27564007565AC756C00756DB4
:10092D00D37571007572FA90E680E030E70E85643C
:10093D0068856569856C6A856D6B800C856C6885CD
:10094D006D6985646A85656BEE54E07003020A710A
:10095D007516007517807E007F908E188F19C374E1
:10096D00209FFF74019ECF2402CF3400FEE48F112F
:10097D008E10F50FF50EF50DF50CF50BF50AAF1103
:10098D00AE10AD0FAC0EAB0DAA0CA90BA80AC3127D
:10099D000C56502AE517250DF582E516350CF58315
:1009AD0074CDF0E4FAF9F8E50D2401F50DEA350CF6
:1009BD00F50CE9350BF50BE8350AF50A80C0E4F5C1
:1009CD000DF50CF50BF50AAF11AE10AD0FAC0EAB6E
:1009DD000DAA0CA90BA80AC3120C565035AE0CAFBC
:1009ED000DE5192FF582E5183EF583E0FDE5172F8E
:1009FD00F582E5163EF583EDF0E4FAF9F8EF240102
:100A0D00F50DEA3EF50CE9350BF50BE8350AF50A5F
:100A1D0080B585166685176774902480FF74003441
:100A2D00FFFEC3E56F9FF56FE56E9EF56EC3E5693D
:100A3D009FF569E5689EF568C3E56B9FF56BE56A03
:100A4D009EF56AC3E5659FF565E5649EF564C3E5AE
:100A5D006D9FF56DE56C9EF56CC3E5729FF572E5C6
:100A6D00719EF571D2E843D82090E668E04409F014
:100A7D0090E65CE0443DF0D2AF90E680E020E105E9
:100A8D00D20E12197A90E680E054F7F0538EF8C228
:100A9D000C300A05120663C20A300C29121BFE50D7
:100AAD0024C20C121A8B20091690E682E030E7045E
:100ABD00E020E1EF90E682E030E604E020E0E41291
:0A0ACD001A33121C00120FAB80C791
:010AD70022FC
:1006630090E6B9E0700302073F1470030207E82421
:10067300FE700302087D24FB700302073914700324
:1006830002073314700302072714700302072D2493
:100693000560030208E9121C0240030208F590E614
:1006A300BBE024FE602C14604724FD601614603107
:1006B30024067066E56690E6B3F0E56790E6B4F06D
:1006C3000208F5E56E90E6B3F0E56F90E6B4F0024C
:1006D30008F5E56890E6B3F0E56990E6B4F0020842
:1006E300F5E56A90E6B3F0E56B90E6B4F00208F541
:1006F30090E6BAE0FF121A5FAA06A9077B01EA494E
:100703004B600DEE90E6B3F0EF90E6B4F00208F51F
:1007130090E6A0E04401F00208F590E6A0E0440171
:10072300F00208F5121BC20208F5121BE60208F5D7
:100733001218390208F5121BB00208F5121C044006
:10074300030208F590E6B8E0247F602B14603C2494
:100753000260030207DEA209E433FF25E0FFA20BD8
:10076300E4334F90E740F0E4A3F090E68AF090E69C
:100773008B7402F00208F5E490E740F0A3F090E6F2
:100783008AF090E68B7402F00208F590E6BCE05420
:100793007EFF7E00E0D3948040067C007D018004D0
:1007A3007C007D00EC4EFEED4F24F6F58274133E83
:1007B300F583E493FF3395E0FEEF24A1FFEE34E6E7
:1007C3008F82F583E0540190E740F0E4A3F090E6D4
:1007D3008AF090E68B7402F00208F590E6A0E044FC
:1007E30001F00208F5121C0640030208F590E6B872
:1007F300E024FE601D240260030208F590E6BAE0DF
:10080300B40105C2090208F590E6A0E04401F00234
:1008130008F590E6BAE0705990E6BCE0547EFF7E9E
:1008230000E0D3948040067C007D0180047C007D41
:1008330000EC4EFEED4F24F6F58274133EF583E48F
:1008430093FF3395E0FEEF24A1FFEE34E68F82F5AC
:1008530083E054FEF090E6BCE05480FF131313547E
:100863001FFFE0540F2F90E683F0E04420F00208CE
:10087300F590E6A0E04401F08078121C08507390D4
:10088300E6B8E024FE60202402706790E6BAE0B484
:100893000104D209805C90E6BAE06402605490E6F9
:1008A300A0E04401F0804B90E6BCE0547EFF7E0064
:1008B300E0D3948040067C007D0180047C007D00B1
:1008C300EC4EFEED4F24F6F58274133EF583E4936C
:1008D300FF3395E0FEEF24A1FFEE34E68F82F5832C
:1008E300E04401F0800C1203C6500790E6A0E044F8
:0908F30001F090E6A0E04480F061
:0108FC0022D9
:03003300021BF6B7
:041BF60053D8EF329F
:101B2500758CE0758AC0E58954F04401F589758E98
:081B350003D28CD2A9D2AF2229
:03000B00020C8D57
:100C8D00C0E0C0F0C083C082C0D075D000C000C02D
:100C9D0001C002C003C004C005C006C007758CE0CA
:100CAD00758AC0D28CE47F607EEAFDFCAB60AA5FE2
:100CBD00A95EA85DC3120C56501DAF60AE5FAD5E50
:100CCD00AC5DE4FAF9F8EF2401F560EA3EF55FE971
:100CDD003DF55EE83CF55DE47F01FEFDFCAB60AAF1
:100CED005FA95EA85DC3120C56700975708275639D
:100CFD0001853E62E47F02FEFDFCAB60AA5FA95E4A
:100D0D00A85DC3120C56700D90E678E04480F0900B
:100D1D00E679E570F0E47F03FEFDFCAB60AA5FA908
:100D2D005EA85DC3120C56700690E679E563F0E49B
:100D3D007F04FEFDFCAB60AA5FA95EA85DC3120C2B
:100D4D0056700690E679E562F0E47F05FEFDFCAB9A
:100D5D0060AA5FA95EA85DC3120C56700790E67875
:100D6D00E04440F0E52C2401FFE4352BFEE4FCFDCE
:100D7D00AB60AA5FA95EA85DC3120C5670097570B1
:100D8D00827563017562F0E52C2402FFE4352BFEBC
:100D9D00E4FCFDAB60AA5FA95EA85DC3120C5670A2
:100DAD000D90E678E04480F090E679E570F0E52C62
:100DBD002403FFE4352BFEE4FCFDAB60AA5FA95EC6
:100DCD00A85DC3120C56700690E679E563F0E52C2C
:100DDD002404FFE4352BFEE4FCFDAB60AA5FA95EA5
:100DED00A85DC3120C56700690E679E562F0E52C0D
:100DFD002405FFE4352BFEE4FCFDAB60AA5FA95E84
:100E0D00A85DC3120C56700990E678E04440F0C21C
:100E1D008CD007D006D005D004D003D002D001D09D
:0C0E2D0000D0D0D082D083D0F0D0E032D2
:100090001201000200000040181618A6000001021C
:1000A00000010A06000200000040010009022700CA
:1000B000010100A0FA0904000003FF000000070589
:1000C0000102400000070586020002000705020247
:1000D00000020009022700010100A0FA0904000043
:1000E00002FF00000007050102400000070586022C
:1000F00040000007050202400000040309040E034B
:1001000051004800590043004300440014035100CB
:100110004800590049004D0047002D0030004800BC
:020120000000DD
:03004300021400A4
:0300530002140094
:10140000021B3D00021B9A00021B8400021B5500B8
:10141000021870000218A70002008F00021C0A00C8
:10142000021C0B00021C0C00021C0D000201220019
:10143000021C0E00021C0F00021C1000021C1100F6
:10144000021C1200021C0A00021C1300021C1400E1
:10145000021C1500021C1600021C1700021C1800BA
:10146000021C1900021C0A00021C0A00021C0A00CD
:10147000021C1A00021C1B00021C1C00021C1D0086
:10148000021C1E00021C1F00021C2000021C210066
:10149000021C2200021C2300021C2400021C250046
:1014A000021C2600021C2700021C2800021C290026
:0814B000021C2A00021C2B00A3
:101A330090E682E030E004E020E60B90E682E030BE
:101A4300E119E030E71590E680E04401F07F147E71
:0C1A5300001217BB90E680E054FEF02269
:101A8B0090E682E044C0F090E681F04387010000CD
:041A9B000000002225
:10197A00300E0990E680E0440AF0800790E680E0A5
:10198A004408F07FDC7E051217BB90E65D74FFF019
:0F199A0090E65FF05391EF90E680E054F7F02273
:021A5F00A907D5
:101A6100AE71AF728F828E83A3E064037017AD01F4
:101A710019ED7001228F828E83E07C002FFDEC3EF8
:091A8100FEAF0580DF7E007F004E
:011A8A002239
:1017BB008E1C8F1D90E600E054187012E51D24015D
:1017CB00FFE4351CC313F51CEF13F51D801590E6D4
:1017DB0000E05418FFBF100BE51D25E0F51DE51CBF
:1017EB0033F51CE51D151DAE1C7002151C4E600556
:0617FB00121A9F80EE228D
:101A9F007400F58690FDA57C05A3E582458370F95A
:011AAF002214
:10177000C106C10802371A00022900000255000004
:10178000025703F7024E0000022600000235000057
:1017900001390101340101450001530001400001FC
:1017A00054000151000161A0C10304590000000070
:0A17B000C100C101C105C104C10759
:101AF300200E0B53227FAD227F801215FD2243223D
:091B030080AD227F801215FD2245
:101B0C00300E0B5322FEAD227F801215FD22432294
:091B1C0001AD227F801215FD22AB
:101AD400300E0E7D017F031215FD90E60174CBF0EC
:0F1AE40022E4FD7F031215FD90E6017443F0220A
:100E390090E6007412F090E60174CBF00000009087
:100E4900E61074A0F000000000000090E612F00027
:100E59000000E490E613F000000090E61474E0F05E
:100E6900000000E490E615F000000090E6047480AC
:100E7900F00000007402F00000007406F0000000A9
:100E8900E4F000000090E60274E6F000000090E64D
:100E99000374F8F000000090E670E04440F00000B0
:100EA90000E490E609F000000043B20F90E6180450
:100EB900F00000007411F000000090E61A7409F0C7
:100EC900000000E490E671F090E672F0C28C75B211
:100ED9000375B6FF75B4BFC2A5D2817522CFC20E04
:100EE900121AF37F647E00121B6DD20E121AF3C21E
:100EF9000290E65EE04408F0000000E490E68DF020
:100F0900D2A3121BFAC20E121B0C7D507F011215BF
:100F1900FD7D227F021215FD7D017F041215FD7DE5
:100F2900017F081215FDE4FD7F101215FD7D647F18
:100F3900201215FD7D1A7F401215FD7DFF7F80125D
:100F490015FD7D807C00E4FF1214B87DFF7C027FD3
:100F5900011214B87D0F7C007F031214B87D1F7C29
:100F6900007F041214B87D1F7C007F051214B87D20
:100F79001F7C007F061214B87D1F7C007F071214A6
:100F8900B8C200C201D20E121AD4C2A4121BEE7B3F
:100F9900F07D037F821219D8E4FB7D017F8212194B
:020FA900D8224C
:100FAB0020060302106E30000BAD24AC237F011220
:100FBB0014B8C20030012AE53AFD7C007F041214FC
:100FCB00B8E53BFD7C007F051214B8E53CFD7C00C9
:100FDB007F061214B8E53DFD7C007F071214B8C2E2
:100FEB0001300518533F075322C7E53F75F008A49E
:100FFB002522F522FD7F801215FDC20530042CAD94
:10100B00497F041215FDAD507F021215FDAD417FD6
:10101B00F01215FDAD427FF11215FDAD437FF212BB
:10102B0015FDAD447FF31215FDC204E55414601297
:10103B0014601A2402702130A6032007FA12155EE1
:10104B00806F30A6032007FA1211CC806430A60300
:10105B002007FA1212A9805930A6032007FA12159D
:10106B005E804EE4FAF9F8E55C2401F55CEA355B49
:10107B00F55BE9355AF55AE83559F559E47F64FEC5
:10108B00FDFCAB5CAA5BA95AA859C3120C567003A2
:10109B00121801E47F207E4EFDFCAB5CAA5BA95AC3
:1010AB00A859D3120C564009E4F55CF55BF55AF5DB
:0910BB0059E551B40102C20622FC
:021BFE00D322F0
:021C0000D322ED
:021C0200D322EB
:1018390090E680E030E71590E6247402F00000009D
:10184900E490E625F0000000D2028013E490E6243B
:10185900F000000090E6257440F0000000C20290FC
:07186900E6BAE0F552D322BC
:101BB00090E740E552F0E490E68AF090E68B04F07E
:021BC000D3222E
:081BE60090E6BAE0F528D322D5
:101BC20090E740E528F0E490E68AF090E68B04F096
:021BD200D3221C
:021C0400D322E9
:021C0600D322E7
:021C0800D322E5
:1003C60090E6B9E0244B606F14700302051E24FC0E
:1003D60070030205A11470030205BF147003020521
:1003E600F724FA700302061D24F970030205562449
:1003F600166003020661E490E68AF090E68BF00050
:10040600000090E6047480F0000000C20E121AF399
:1004160090E6047406F0000000E4F0FF7E01121777
:10042600BBD20E121AF37F0A7E001217BB75250186
:10043600C203D206020661E490E68AF090E68BF0EB
:1004460090E6A0E020E1F990E68BE0F51AE4F51BD2
:100456007440251BF582E434E7F583E0FF7400253C
:100466001BF582E43428F583EFF0051BE51BB44049
:10047600DF902807E0FD7F401215FD902808E0FD7B
:100486007F201215FD902811E0FD7F101215FD90BA
:100496002812E0FD7F081215FD902820E0F5459012
:1004A600282EE0F54090283AE0F56190283CE0F5EA
:1004B60054A3E0F551902821E0FF70035322BFEFCB
:1004C600B401035322BFEFB402035322BFEFB403B8
:1004D6000343224090282AE070055322FD800343FF
:1004E6002202AD227F801215FDAD617F011215FD3E
:1004F6007D0F7C007F031214B87D807C00E4FF1220
:1005060014B890283BE07008C20E121AD402066195
:10051600D20E121AD4020661E4F51B7400251BF5EF
:1005260082E43428F583E0FF7440251BF582E43429
:10053600E7F583EFF0051BE51BB440DF000000E4A0
:1005460090E68AF000000090E68B7440F0020661A7
:10055600E490E68AF090E68BF090E6A0E020E1F9E0
:1005660090E68BE0F51A90E740E054F0FFC4540F94
:1005760024F0FB7D017F821219D890E741E075F0E7
:100586000AA4FFAEF01217BB90E740E024F0540F28
:10059600FB7D017F821219D8020661E490E68AF09B
:1005A60090E68BF090E6A0E020E1F990E68BE0F58E
:1005B6001A000000C206020661E490E68AF090E6A0
:1005C6008BF090E6A0E020E1F990E68BE0F51A00CA
:1005D600000090E740E0F546A3E0FEA3E07C00249F
:1005E60000F548EC3EF547AD48FCAF461214B8801E
:1005F6006AE490E68AF090E68BF090E6A0E020E1CF
:10060600F990E68BE0F51A00000090E740E0FFA3C2
:10061600E0FD1215FD804490E74074B1F0A374111B
:10062600F0A37403F0A3741BF0A37402F0A3745434
:10063600F0A37401F0A304F0A374B8F0300205E44B
:10064600A3F0800690E74974FFF0000000E490E60E
:0C0656008AF000000090E68B740AF0C3EC
:010662002275
:101B3D00C0E0C083C082D20A5391EF90E65D74017C
:081B4D00F0D082D083D0E03219
:101B8400C0E0C083C0825391EF90E65D7404F0D04E
:061B940082D083D0E03294
:101B9A00C0E0C083C0825391EF90E65D7402F0D03A
:061BAA0082D083D0E0327E
:10187000C0E0C083C08290E680E030E70E856468F7
:10188000856569856C6A856D6B800C856C68856D76
:101890006985646A85656B5391EF90E65D7410F01D
:0718A000D082D083D0E032BA
:101B5500C0E0C083C082D20C5391EF90E65D74085B
:081B6500F0D082D083D0E03201
:1018A700C0E0C083C08290E680E030E70E856468C0
:1018B700856569856C6A856D6B800C856C68856D3F
:1018C7006985646A85656B5391EF90E65D7420F0D6
:0718D700D082D083D0E03283
:01008F00323E
:011C0A0032A7
:011C0B0032A6
:011C0C0032A5
:011C0D0032A4
:10012200C0E0C0F0C083C082C0D075D000C000C0A3
:0D01320001C002C003C004C005C006C00724
:10013F00C2AF90E6A1E020E1F990E780E0FF120C5A
:10014F0067017B00019B0101E10201F703020E042D
:10015F00026C05028006028B0702AA08036D0901D3
:10016F0096FD018BFE0181FF0000039775250002AC
:10017F000397752500D203C20602039790E781E02B
:10018F0024FF9207020397C28C020397000000908E
:10019F00E6047480F00000007406F0000000E4F044
:1001AF00E53AFD7C007F041214B8E53BFD7C007F2F
:1001BF00051214B8E53CFD7C007F061214B8E53D2E
:1001CF00FD7C007F071214B8752501C203D2060209
:1001DF00039790E781E0FEA3E07C002400F524EC78
:1001EF003EF523D20002039790E781E0F53AA3E0B2
:1001FF00F53BA3E0F53CA3E0F53DD2010203979058
:10020F00E781E0F52DA3E0F52FA3E0F52EAF2FE466
:10021F00FCFDFEFB7A01F9F8120B39C004C005C0D2
:10022F0006C007AF2DE4FCFDFEFBFA7901F8120BB7
:10023F0039D003D002D001D000EF2BFBEE3AFAED0C
:10024F0039F9EC38F8E4FCFDFEEB252EF533EE3AE8
:10025F00F532ED39F531EC38F53002039790E7813F
:10026F00E0FEA3E07C002400F536EC3EF5350203FA
:10027F009790E781E0F53FD20502039790E781E081
:10028F00F549A3E0F550A3E0F541A3E0F542A3E063
:10029F00F543A3E0F544D204020397E4FF74802FE3
:1002AF00F582E434E7F583E0FE74002FF582E43441
:1002BF0028F583EEF00FBF40E4902807E0FD7F4064
:1002CF001215FD902808E0FD7F201215FD902811D2
:1002DF00E0FD7F101215FD902812E0FD7F0812152A
:1002EF00FD902820E0F54590282EE0F54090283A23
:1002FF00E0F56190283CE0F554A3E0F551902821FA
:10030F00E0FF70035322BFEFB401035322BFEFB4DA
:10031F0002035322BFEFB4030343224090282AE085
:10032F0070055322FD8003432202AD227F801215F8
:10033F00FDAD617F011215FD7D0F7C007F0312144F
:10034F00B87D807C00E4FF1214B890283BE0700762
:10035F00C20E121AD48031D20E121AD4802AD28C25
:10036F0090E781E0540FF53EA3E0FEA3E07C00246C
:10037F0000FFEC3EC313F52BEF13F52C75600075E2
:10038F005F00755E00755D0000000090E68DE4F083
:0C039F005391EF90E65FE04408F0D2AF0D
:1003AB00D007D006D005D004D003D002D001D000A6
:0B03BB00D0D0D082D083D0F0D0E03250
:011C0E0032A3
:011C0F0032A2
:011C100032A1
:011C110032A0
:011C1200329F
:011C1300329E
:011C1400329D
:011C1500329C
:011C1600329B
:011C1700329A
:011C18003299
:011C19003298
:011C1A003297
:011C1B003296
:011C1C003295
:011C1D003294
:011C1E003293
:011C1F003292
:011C20003291
:011C21003290
:011C2200328F
:011C2300328E
:011C2400328D
:011C2500328C
:011C2600328B
:011C2700328A
:011C28003289
:011C29003288
:011C2A003287
:011C2B003286
:101B6D00AD07AC06ED25E0FDEC33FCED4C6007ED6B
:071B7D001D70011C80F52220
:10168200C2A4E545B40105D20E121B0C752501E575
:101692002D75F040A485F01AF51BAF257E00AC1A1B
:1016A200AD1B120B27D3EF9400EE940040117FDEA6
:1016B2007E031217BBE51B151B7002151A80DB7522
:1016C2001A00852F1BAF257E00AC1AAD1B120B270B
:1016D200D3EF9400EE940040117FFD7E001217BB01
:1016E200E51B151B7002151A80DBAF2E7E00121748
:0D16F200BBE545B40105C20E121B0CC2A4DD
:0116FF0022C8
:041BFA0075B1EE22B1
:1018010075B1EE00000075B16E00000075B16F009A
:10181100000075B16D00000075B17D000000000091
:101821000075B17C00000075B1EC00000075B1EEEF
:08183100000000D2A7D2A7229B
:1019A90075B16E00000075B16F00000075B16D0072
:1019B900000075B17D00000075B17C00000075B1B3
:0F19C900EC00000075B1EEC2A7000000D2A7220B
:101BD400E4FFFE1218010FBF00010EBE01F5BFF8AD
:011BE400F20E
:011BE50022DD
:1017000075B1EE00000075B16E00000000000075BC
:10171000B16A75B16B00000000000075B14B0000AC
:101720000000000075B14F00000000000075B16FAF
:1017300000000000000000000075B16D0000000016
:10174000000075B17D00000000000075B17C000054
:101750000000000075B1FC00000000000075B1EC55
:1017600000000000000075B1EE0000000000002243
:0F008000C2A77F037E00121B6DD2A7121B6D2239
:0614B8008C1C8D1DA9072C
:1014BE00530107C2A37F0A7E00121B6DC2A2121B2C
:1014CE006DD2A1121B6DC2A1E4FBFAAF03E9A8070E
:1014DE00088002C313D8FC30E004D2A28002C2A25C
:1014EE007F0A7E00121B6DD2A1121B6DC2A1121BB0
:1014FE006D0BBB00010AEB64034A70CFC2A27F0AD8
:10150E007E00121B6DD2A1121B6DC2A1E4FAFBAFBD
:10151E0003E51DAE1CA807088005CEC313CE13D855
:10152E00F930E004D2A28002C2A27F0A7E00121B12
:10153E006DD2A1121B6DC2A1121B6D0BBB00010A55
:0F154E00EB640B4A70C9D2A37F0A7E00121B6D9B
:01155D00226B
:0415FD008F1CA90591
:10160100C2A07F017E00121B6DE4FBFAAF03E9A8C3
:1016110007088002C313D8FC30E004D2A28002C2C2
:10162100A27F017E00121B6DD2A1121B6DC2A112FD
:101631001B6D0BBB00010AEB64084A70CFE4FAFB97
:10164100AF03E51CA807088002C313D8FC30E004EF
:10165100D2A28002C2A27F017E00121B6DD2A11212
:101661001B6DC2A1121B6D0BBB00010AEB64084A82
:1016710070CED2A07F017E00121B6DC2A0121B6D25
:011681002246
:1019D800AC07AA0590E678E04480F090E679ECF050
:1019E8007F647E00121B6DEAF0121B6DEBF0121B78
:0E19F8006D90E678E04440F07F64121B6D2293
:101AB00090282AE07019432202AD227F801215FD82
:101AC000D2A5C2A55322FDAD227F801215FD22D2E0
:041AD000A5C2A522E4
:10155E0085334D85324C85314B85304AE4FFFEE5AF
:10156E004BFDE4FCFB7A01F9F8120BC4E4FB7A01A3
:10157E00F9F8120BC48F2DE4FFE54CFEE4FDFCFBE5
:10158E007A01F9F8120BC48F2FE54DFFE48F2E125E
:10159E001AB0121682E4FFFEFDFCAB4DAA4CA94B0D
:1015AE00A84AD3120C564003121BD4121700E4FBA8
:1015BE00FAC3EB940AEA648094805004D2808002CD
:1015CE00C280C2817F017E00121B6D208303300317
:1015DE00FAD281EBB53609EAB535051219A98003A1
:0E15EE001218010BBB00010ABA01C6BBF8C3FC
:0115FC0022CC
:1011CC0085334D85324C85314B85304AE47F03FEA7
:1011DC00FDFCAB4DAA4CA94BA84AC3120C565005AA
:1011EC00755301801BE54D24FDF54DE54C34FFF5A1
:1011FC004CE54B34FFF54BE54A34FFF54AE4F55327
:10120C00E4FFFEE54BFDE4FCFB7A01F9F8120BC49C
:10121C00E4FB7A01F9F8120BC48F2DE4FFE54CFEC8
:10122C00E4FDFCFB7A01F9F8120BC48F2FE54DFF9E
:10123C00E48F2EE553B40103121BD4121AB0120022
:10124C008075B1FF121682E5537003121BD412176E
:10125C0000D280E545B401057F64121A06C280E510
:10126C0045B401057F64121A06E4FBFAC3EB940A39
:10127C00EA648094805004D2808002C280C2817F54
:10128C00017E00121B6D2083033003FAD2811218E9
:0C129C00010BBB00010ABA01D3BBF8D063
:0112A8002223
:1012A90085334D85324C85314B85304AE4FFFEE567
:1012B9004BFDE4FCFB7A01F9F8120BC4E4FB7A015B
:1012C900F9F8120BC48F2DE4FFE54CFEE4FDFCFB9D
:1012D9007A01F9F8120BC48F2FE54DFFE48F2E1216
:1012E9001AB0121682E4FFFEFDFCAB4DAA4CA94BC5
:1012F900A84AD3120C564003121BD4121700E4FB60
:10130900FA1218010BBB00010AEB64664A70F2E499
:10131900FAFBC3EB940AEA648094805004D280807B
:1013290002C280C2817F0A7E00121B6D20830330B6
:1013390003FAD281EBB53609EAB535051219A98048
:10134900031218010BBB00010ABA01C6BB2CC3E486
:10135900FAFB1218010BBB00010AEB64664A70F232
:011369002261
:101A06008F1A5322FBAD227F801215FDE51A601254
:101A1600C2817F0A7E00121B6D3083FDD281151AAA
:0D1A260080EA432204AD227F801215FD22CC
:081BEE00E4F578D2E9D2AF2240
:1018DE0090E678E020E6F9C2E990E678E04480F000
:1018EE00EF25E090E679F090E678E030E0F990E6CA
:1018FE0078E04440F090E678E020E6F990E678E073
:06190E0030E1D6D2E9220F
:10194800A90790E678E020E6F9E578702390E67834
:10195800E04480F0E925E090E679F08D73AF03A9C3
:10196800077574018A758976E4F577757801D3224D
:02197800C32288
:10191400A90790E678E020E6F9E578702590E67866
:10192400E04480F0E925E0440190E679F08D73AF5E
:1019340003A9077574018A758976E4F577757803C8
:04194400D322C322C5
:03004B000210C4DC
:1010C400C0E0C083C082C085C084C086758600C06D
:1010D400D075D000C000C001C002C003C006C00764
:1010E40090E678E030E2067578060211AE90E67874
:1010F400E020E10CE578640260067578070211AE21
:10110400E57824FE605F14603624FE700302119FAC
:1011140024FC70030211AB240860030211AEAB740B
:10112400AA75A976AF7705778F82758300120AD8DE
:1011340090E679F0E57765737070757805806B904B
:10114400E679E0AB74AA75A976AE778E82758300D2
:10115400120B05757802E5736401704E90E678E031
:101164004420F08045E57324FEB5770790E678E0E7
:101174004420F0E57314B5770A90E678E04440F033
:1011840075780090E679E0AB74AA75A976AE778E8F
:1011940082758300120B050577800F90E678E04492
:1011A40040F075780080037578005391DFD007D044
:1011B40006D003D002D001D000D0D0D086D084D0C5
:0811C40085D082D083D0E03217
:0300000002136A7E
:0C136A00787FE4F6D8FD7581780213B19D
:100AD800BB010CE58229F582E5833AF583E02250D3
:100AE80006E92582F8E622BBFE06E92582F8E2221D
:0D0AF800E58229F582E5833AF583E4932237
:100B0500F8BB010DE58229F582E5833AF583E8F026
:100B1500225006E92582C8F622BBFE05E92582C8D2
:020B2500F222BA
:100B2700EF8DF0A4A8F0CF8CF0A428CE8DF0A42EE2
:020B3700FE229C
:100B3900E88FF0A4CC8BF0A42CFCE98EF0A42CFC5B
:100B49008AF0EDA42CFCEA8EF0A4CDA8F08BF0A4D9
:100B59002DCC3825F0FDE98FF0A42CCD35F0FCEB38
:100B69008EF0A4FEA9F0EB8FF0A4CFC5F02ECD39FD
:0F0B7900FEE43CFCEAA42DCE35F0FDE43CFC226A
:100B880075F008758200EF2FFFEE33FECD33CDCC24
:100B980033CCC58233C5829BED9AEC99E5829840A7
:100BA8000CF582EE9BFEED9AFDEC99FC0FD5F0D684
:100BB800E4CEFBE4CDFAE4CCF9A88222B800C1B9AE
:100BC8000059BA002DEC8BF084CFCECDFCE5F0CBEC
:100BD800F97818EF2FFFEE33FEED33FDEC33FCEB25
:100BE80033FB10D703994004EB99FB0FD8E5E4F9E0
:100BF800FA227818EF2FFFEE33FEED33FDEC33FCCD
:100C0800C933C910D7059BE99A4007EC9BFCE99AC0
:100C1800F90FD8E0E4C9FAE4CCFB2275F010EF2F05
:100C2800FFEE33FEED33FDCC33CCC833C810D70705
:100C38009BEC9AE899400AED9BFDEC9AFCE899F840
:0E0C48000FD5F0DAE4CDFBE4CCFAE4C8F922D3
:100C5600EB9FF5F0EA9E42F0E99D42F0E89C45F0F4
:010C6600226B
:100C6700D083D082F8E4937012740193700DA3A31C
:100C770093F8740193F5828883E473740293686030
:060C8700EFA3A3A380DF30
:101376000208FDE493A3F8E493A34003F68001F288
:1013860008DFF48029E493A3F85407240CC8C33378
:10139600C4540F4420C8834004F456800146F6DF47
:1013A600E4800B0102040810204080901770E47E50
:1013B600019360BCA3FF543F30E509541FFEE4933C
:1013C600A360010ECF54C025E060A840B8E493A303
:1013D600FAE493A3F8E493A3C8C582C8CAC583CA2E
:1013E600F0A3C8C582C8CAC583CADFE9DEE780BEE6
:0117BA00002E
:00000001FF
